:10F000004BC0000075C0000073C0000071C000005C
:10F010006FC000006DC000006BC0000069C0000040
:10F0200067C0000065C0000000C2000061C00000B1
:10F030005FC000005DC000005BC0000059C0000060
:10F0400057C0000055C0000053C0000051C0000070
:10F050004FC000004DC000004BC0000049C0000080
:10F0600047C0000045C0000043C0000041C0000090
:10F070003FC000003DC000003BC0000039C00000A0
:10F0800037C0000035C0000033C0000031C00000B0
:10F090002FC000002DC0000011241FBECFEFD0E113
:10F0A000DEBFCDBF04B603FE0EC080915401909127
:10F0B000550182349C4D39F410925501109254013F
:10F0C000E0E0F0E0099511E0A0E0B1E0E0EDF7EF5D
:10F0D00002C005900D92AA34B107D9F721E0AAE445
:10F0E000B1E001C01D92A435B207E1F702D06EC3B2
:10F0F00087CF84B7877F84BF88E10FB6F894809369
:10F100006000109260000FBE81E085BF82E085BF85
:10F1100071D1789480910001882311F03CD3FACF0B
:10F120008091E00081608093E00082E49CED909308
:10F130005501809354012CE088E190E00FB6F894DB
:10F14000A895809360000FBE20936000FFCF42E33C
:10F1500061EC81E0DCC080914C018F77813209F055
:10F160005DC080914D01893009F058C08091E80060
:10F17000877F8093E8008091E80082FFFCCF309188
:10F18000F1002091F100832F922F8F3F2FEF9207F4
:10F1900019F41092000132C023E0FC0120935700C3
:10F1A000E89507B600FCFDCF20E030E061E040913B
:10F1B000F2005091F300452B39F1E091F10070918C
:10F1C000F1004E2F572FF901EE0FFF1FE80FF91F27
:10F1D0000A0160935700E89511242F5F3F4F2038B4
:10F1E000310529F725E0FC0120935700E89507B683
:10F1F00000FCFDCF81E180935700E8958091E80005
:10F200008B778093E80097C04091E8004B7740935C
:10F21000E8004091E80042FFFCCFCFCF0895913045
:10F2200049F0923061F0913279F489E090E023E185
:10F2300031E00EC082E190E023E231E009C082E2D9
:10F2400090E021E031E004C085E190E025E331E089
:10F25000FA013183208308952091520130915301A6
:10F260002617370748F06115710539F42091E80039
:10F270002E772093E80001C0B901FC0120E0611560
:10F28000710591F18EB38823E1F18530E1F1809130
:10F29000E80083FD3AC08091E80082FF06C08091BB
:10F2A000E80082FF24C080E008958091E80080FF9C
:10F2B000E6CF8091F2009091F3006115710551F055
:10F2C0008830910538F421912093F1006150710943
:10F2D0000196F3CF21E0089709F020E08091E80043
:10F2E0008E778093E800CBCF2111CCCFD8CF8EB3CF
:10F2F000882339F0853039F08091E80083FFCFCF43
:10F3000004C082E0089583E0089581E008958F703D
:10F310008093E900EBEEF0E0808181608083EDEE88
:10F32000F0E010826093EC0040838091EE00881F33
:10F330008827881F089580914C0187FD05C0809122
:10F34000E80080FF0DC010C08091E80082FD04C07D
:10F350008EB38111F9CF08958091E8008B7707C0B3
:10F360008EB38111ECCF08958091E8008E77809361
:10F37000E80008950F931F93CF93DF9349D050D0A7
:10F38000C8EDD0E088818F77888388818068888302
:10F3900088818F7D8883E7EDF0E0808180688083BD
:10F3A00019BC1EBA10924A0100EE10E0F8018081EB
:10F3B0008B7F808388818160888342E060E080E089
:10F3C000A6DFE1EEF0E080818E7F8083E2EEF0E068
:10F3D000808181608083808188608083F801808162
:10F3E0008E7F8083888180618883DF91CF911F9198
:10F3F0000F910895E8EDF0E080818F7E8083E7ED46
:10F40000F0E080818160808381E080934B01B2CF06
:10F41000E8EDF0E080818C7F80831092E200089517
:10F420001092DA001092E10008951F920F920FB629
:10F430000F9211242F933F934F935F936F937F937A
:10F440008F939F93AF93BF93EF93FF938091DA00D5
:10F4500080FF1BC08091D80080FF17C08091DA0028
:10F460008E7F8093DA008091D90080FF0BC08CE002
:10F4700089BD8EE089BD09B400FEFDCF81E08EBB61
:10F4800089D103C019BC1EBA85D18091E10080FFEB
:10F4900017C08091E20080FF13C08091E2008E7F50
:10F4A0008093E2008091E20080618093E20080918D
:10F4B000D80080628093D80019BC85E08EBB6AD1E9
:10F4C0008091E10084FF2EC08091E20084FF2AC079
:10F4D0008CE089BD8EE089BD09B400FEFDCF80912E
:10F4E000D8008F7D8093D8008091E1008F7E80933B
:10F4F000E1008091E2008F7E8093E2008091E20043
:10F5000081608093E20080914A01882311F084E0B9
:10F5100007C08091E30087FF02C083E001C081E063
:10F520008EBB38D18091E10083FF21C08091E20041
:10F5300083FF1DC08091E100877F8093E10082E01E
:10F540008EBB10924A018091E1008E7F8093E10092
:10F550008091E2008E7F8093E2008091E2008061E2
:10F560008093E20042E060E080E0D1DE13D1FF91C1
:10F57000EF91BF91AF919F918F917F916F915F912B
:10F580004F913F912F910F900FBE0F901F901895A4
:10F590001F93CF93DF9300D0CDB7DEB7ECE4F1E05B
:10F5A0008091F100819381E0E435F807C9F7D3DD5C
:10F5B0008091E80083FFDAC090914C0180914D0169
:10F5C000853009F465C030F4813059F168F083303A
:10F5D00041F1CCC0883009F49CC0893009F4ABC03B
:10F5E000863009F0C3C075C0903881F0923809F0B8
:10F5F000BDC0809150018F708093E9009091EB0025
:10F6000095FB992790F91092E90001C090E0809154
:10F61000E800877F8093E8009093F1001092F1005A
:10F6200083C0292F2D7F09F0A1C0923009F09EC020
:10F6300090914E01911126C0209150012F7009F434
:10F6400095C02093E9009091EB0090FF1BC08330A0
:10F6500021F48091EB00806213C08091EB00806107
:10F660008093EB0081E090E0022E01C0880F0A94A5
:10F67000EAF78093EA001092EA008091EB0088603C
:10F680008093EB001092E9008091E800877F4FC0E3
:10F6900091116CC010914E011F778091E30080782A
:10F6A000812B8093E3008091E800877F8093E800BE
:10F6B00042DE8091E80080FFFCCF8091E30080680B
:10F6C0008093E300112311F083E001C082E08EBB40
:10F6D0004DC09058923008F049C0AE014F5F5F4F67
:10F6E0006091500180914E0190914F0198DD0097FB
:10F6F00009F43CC02091E800277F2093E800BC017A
:10F7000089819A81A9DD8091E8008B778093E80058
:10F710002DC0903859F58091E800877F8093E800EC
:10F7200080914A018093F1008091E8008E77809368
:10F73000E80001DE1BC0911119C090914E0192307A
:10F74000A8F48091E800877F8093E80090934A01B5
:10F75000F2DD80914A01811104C08091E30087FFAE
:10F7600002C084E001C081E08EBBF1DC8091E80042
:10F7700083FF0AC08091E800877F8093E800809132
:10F78000EB0080628093EB000F900F90DF91CF91A0
:10F790001F9108950895CF938EB38823A9F0809187
:10F7A000E9008F709091EC0090FF02C090E801C0DA
:10F7B00090E0C92FC82B1092E9008091E80083FDEA
:10F7C000E7DECF70C093E900CF910895F894FFCFA2
:10F7D0000109022200010100803209040000010336
:10F7E0000000000921110100012215000705810315
:10F7F0004000051201100100000008EB0367200122
:10F80000000000000106DCFF09FBA1010902150050
:0AF8100025FF75089602019102C061
:040000030000F00009
:00000001FF
